:10000000A3C0FDC1BBC0BAC0B9C0B8C0B7C0B6C0FC
:10001000B5C0B4C0B3C0B2C0B1C0B0C0AFC0AEC054
:10002000ADC0ACC0ABC009022200010100803C0998
:100030000400000103000000092101010001220069
:10004000000705810308000A04030904180372006D
:100050006100700068006E00650074002E006E0084
:1000600065007400140334006E00650073003400F2
:1000700073006E00650073000A0331003000300029
:10008000300005010904A1010901A1008501093021
:100090000931150026FF007508950281020509192E
:1000A00001290815002501750195088102C0C005C8
:1000B000010904A1010901A10085020930093115D6
:1000C0000026FF007508950281020509190129081B
:1000D00015002501750195088102C0C005010904BC
:1000E000A1010901A100850309300931150026FF8E
:1000F00000750895028102050919012908150025D6
:1001000001750195088102C0C005010904A101091A
:1001100001A100850409300931150026FF0075088A
:1001200095028102050919012908150025017501AB
:1001300095088102C0C0120101010000000881176A
:100140009D0A01010102030111241FBECFE5D4E085
:10015000DEBFCDBF10E0A0E6B0E0E0E5FCE002C00D
:1001600005900D92A637B107D9F710E0A6E7B0E0E9
:1001700001C01D92AD3DB107E1F749C341CF86E70C
:1001800090E08093D1000B968093C50085B7836083
:1001900085BF8BB780648BBF08951F93DC01162F3A
:1001A000693008F018E090918E0090FF02C023ECB7
:1001B00001C02BE48091620087FF04C09F5F909391
:1001C0008E0003C08FEF809362002093C600912FB2
:1001D000E7ECF0E002C08D9181939150E0F7612F40
:1001E00087EC90E0BED21C5F109362001F910895CF
:1001F0000F931F938091D600882309F496C0982FFF
:10020000935097FD90C0E6E7F0E08091C500E82F9D
:10021000EF5F8091D3008D3209F07FC0983009F0F4
:100220007CC08081807609F074C01092C00081810A
:10023000882321F41092C10022E05CC0853021F4B3
:1002400082818093D70055C08630F1F5838181305B
:1002500039F42091D8008091C3009091C40032C03D
:10026000823021F486E290E022E22CC08330C9F48F
:100270008281882321F488E490E024E023C0813047
:1002800021F48CE490E028E11DC0823021F484E662
:1002900090E024E117C0833061F488E790E02AE021
:1002A00011C0813221F488E390E029E00BC0823252
:1002B00019F020E030EC1FC02091C2008091DB00DB
:1002C0009091DC0030EC19C0883029F421E030E84E
:1002D0008AED90E012C0893021F482818093DA00A7
:1002E00008C08A3011F421E005C08B3011F410925F
:1002F0008E0020E030E880EC90E09093D500809371
:10030000D4008781882359F48681821740F4282FEE
:1003100006C0CF012AD2282F01C020E030E8309358
:100320008C00209360001092D600909160009F3F57
:1003300009F44BC08091610087FF47C0692F993055
:1003400008F068E0961B9093600080918C0080FF1D
:1003500002C003EC01C00BE48F5F80938C00E0913E
:10036000D400F091D50086FD04C0962FA8EBB0E034
:1003700017C04091C200262FA8EBB0E00CC034910A
:10038000CD01019650E0EF33F50711F44C9301C015
:100390003C93DC013196215090F704C081918D93FC
:1003A0009150E0F7F093D500E093D4007727162F13
:1003B00088EB90E0D6D1183018F48FEF809360006E
:1003C0000093B7001C5F1093610080B3857019F033
:1003D00010928D0011C080918D00882369F494E6FD
:1003E00080B3857049F49150D9F781E080938D00F6
:1003F0001092D7001092D2001F910F9108950F9381
:100400000FB70F93809BFECF809B06C0809B04C0DC
:10041000809B02C0000000C01F933F932F9331E0E8
:1004200014E000B3102710FD32E0102F3A95C9F701
:1004300000FDE7C000B3102717952FE72795DF933E
:1004400010B3012707952795CF93C091D10000B332
:100450001027179527953BE0D0E04F9310B3012765
:10046000079527954FEF000055C0809BFECF809BDE
:1004700006C0809B04C0809B02C0000000C0DF91CA
:1004800000C0CDCF10B3157079F1407C2C6F13C034
:1004900000B3057049F141782C6F15C0057021F14A
:1004A000102F2C6F00B319C000B30570E9F04E7F18
:1004B0002C6F18C038F300B30570B1F010271795F2
:1004C0002795243028F310B3012707952795422755
:1004D00049934FEF00B3243008F310271795279561
:1004E000243010F310B31570E1F10127079527951B
:1004F0002430F0F000B30570A1F11027179527956F
:100500002430E0F010B30127079527953A9541F183
:100510002430D0F000B3057021F1102717952795EE
:100520002430C0F010B30127079527952430C2CF9F
:1005300010B31570B1F04C7F2C6FDCCF00B3057099
:1005400081F0487F2C6FDECF10B3157051F0407FE3
:100550002C6FE0CF00B3057021F0407E2C6FE2CF0E
:100560003DC03C2FC091D1003C1B00E433300ABF9A
:10057000A8F108811981412F1F772091D2000D32F7
:1005800089F1013E79F10936C1F00777033431F57D
:100590001091D900112311F10091D6000030D1F54E
:1005A0003430DAF13093D6001093D3000091C500B7
:1005B000C093C5000093D10030C0121779F447FDF5
:1005C0003AC0309161003F3F29F10FEF0093610085
:1005D000C7EBD0E025C000270093D9004F91CF9101
:1005E000DF910FC01217B9F70093D9000FEF0093F6
:1005F0006000009361004F91CF910AB706FD35CF9F
:10060000DF9100E40ABF2F913F911F910F910FBF1F
:100610000F911895C4E6D0E002C0C3E6D0E032E006
:100620005F9302B30A7F016002BB55E011B315600E
:1006300011BB20E819C0309162003F3F59F30FEF22
:1006400000936200C6ECD0E0EBCF052710E002BBC0
:1006500010C0052710E0089402BB13C0052710E066
:1006600015C0052710E019C020FF052702BB2795FC
:1006700017951C3F50F720FF0527279502BB1795BC
:100680001C3F38F720FF05272795179502BB1C3F15
:1006900028F720FF0527279517951C3F02BB08F771
:1006A00000C0499120FF052702BB279517951C3FE5
:1006B00080F520FF0527279502BB17951C3F68F59D
:1006C00020FF05272795179502BB1C3F58F520FFF3
:1006D0000527279517951C3F02BB38F5242F3A951F
:1006E00019F60A7F5F9102BB32E03A95F1F710915B
:1006F000D700C656D04011F01093D200016011B35C
:100700001A7F02BB0A7F4F91CF9111BB02BBDF91D1
:1007100078CF052710E002BBCACF052710E0089468
:1007200002BBCDCF052710E0CFCF052710E0D3CFF8
:10073000A82FB92F8FEF9FEF41E050EA615070F082
:100740002D9138E0722F782796958795269570FF22
:1007500002C0842795273A95A9F7F0CF8095909508
:100760000895E6DF8D939D930895CF93DF93DC0189
:1007700022E930E03093D5002093D4008C9180762C
:10078000803209F03FC0ED018981823091F08A30DA
:1007900009F18130B9F510928F00E0919000F0914D
:1007A00091000784F089E02D6A81C9010995992794
:1007B0002BC0FD019281892F8150883018F5892F37
:1007C000992783569F4F9093D5008093D40081E062
:1007D00090E01AC0ED01EA81EE2351F4EEE9F0E079
:1007E000ED018B81819380E0E63AF80759F0F8CF6C
:1007F0008E2F8150883030F4FF27E356FF4FED01F4
:100800008B81808380E090E0DF91CF910895C7E5F0
:10081000D4E0DEBFCDBF88E0FE01319611928A950B
:10082000E9F773D1FC01909391008093900083814C
:1008300094819093DC008093DB0081818093C200DF
:1008400087819085009731F09093C4008093C30016
:10085000858107C086E391E09093C4008093C30034
:10086000E7D18093D80014BA8FEF85BB88EF82BBA5
:1008700085E081BB9EEF8FEF9150F1F78150E1F75A
:1008800011BA85E083BF8FE085BD84EC83BDE09124
:100890009000F09191000184F285E02D09956FDCC4
:1008A000E0919000F09191000384F485E02D09958A
:1008B0007894FF24A8959CDC08B607FE2BC080E83E
:1008C00088BFE0919000F09191000384F485E02DC1
:1008D000099500E010E013C00584F685E02D802F17
:1008E0008F5F0995882349F081E090E0002E02C0D7
:1008F000880F991F0A94E2F7F82A0F5F1F4FE091C3
:100900009000F09191008081992787FD90950817BC
:10091000190714F308B600FE2FC081E088BF40918C
:1009200090005091910020E030E00EE910E0FE01CF
:10093000319661E070E018C0D8019C91992379F05C
:100940008081853018F08550808309C09083CB0169
:10095000022E02C0880F991F0A94E2F7F82A2F5F2F
:100960003F4F0F5F1F4F3196DA018C91992787FD1A
:1009700090952817390704F3FF2009F49BCF00E076
:1009800010E025C08F2D992787FD9095002E02C07D
:10099000959587950A94E2F780FF17C080916200D1
:1009A0008F3F99F4602F6F5F0784F089E02D82E913
:1009B00090E00995682F82E990E0EFDB02C018DC37
:1009C000A895809162008F3FD1F70F5F1F4FE09194
:1009D0009000F09191008081992787FD90950817EC
:1009E000190784F266CFAC9A80E38A95F1F7AC9848
:1009F00020E030E040E050E060E070E098E1892FD6
:100A00008A95F1F7AD98440F550F660F770F9B9BB2
:100A100041609A9B5160999B6160989B7160892F9E
:100A20008A95F1F7AD9A2F5F3F4F2830310539F79E
:100A30004093A7005093A9006093AB007093AD0062
:100A400020E030E098E1892F8A95F1F7AD9846953E
:100A50005695669576959B9B40689A9B5068999BA6
:100A60006068989B7068892F8A95F1F7AD9A2F5F1F
:100A70003F4F2830310539F78091A600992780FD36
:100A800040E04093A80081FD50E05093AA0082FD11
:100A900060E06093AC0083FD70E07093AE00089559
:100AA0001F931FB7F894A49AA59A84B3807F84BB40
:100AB00085B38F6085BBAD9AAC981092A60093DF8A
:100AC0008091A8008F3F19F481E08093A600809167
:100AD000AA008F3F29F48091A60082608093A6002F
:100AE0008091AC008F3F29F48091A60084608093B0
:100AF000A6008091AE008F3F29F48091A600886007
:100B00008093A6001FBF1F91089582E890E0909304
:100B100069008093680085E690E008951F93DC01EA
:100B2000653018F080E090E06FC0162F1150892BCF
:100B300009F459C06C93612F772767FD7095AB015D
:100B4000440F551FFA01E955FF4F8081992780FF17
:100B500002C03FEF01C030E881FD30E0FD0131838C
:100B6000FA01E955FF4F8081992782FF02C03FEFCC
:100B700001C030E883FD30E0FD0132838091A600A2
:100B8000992702C0959587956A95E2F7FA01E9558C
:100B9000FF4F80FF03C08081807F23C020813327E7
:100BA000A901440F452F441F550B5195C90180746D
:100BB000907065E0959587956A95E1F7482BC90196
:100BC0008072907053E0959587955A95E1F7482B80
:100BD0002071307035952795422B81818295807FD9
:100BE000842BFD018383E12FFF27E7FDF095EE0FB6
:100BF000FF1FDF01A955BF4F8D919C91E155FF4F1C
:100C00009183808384E090E01F910895815099271B
:100C100087FD9095880F991FBC0161557F4F42E079
:100C200050E089559F4F07D0992787FD90950895EB
:100C300082E190E00895FB01DC0104C08D910190F8
:100C4000801921F441505040C8F7881B990B089532
:100C5000FFFFFFD25A04B40000000000000050055E
:060C6000F30406068E05F8
:00000001FF
